:0200000480007A
:1000000097170000938707001304F0FF7310043460
:10001000F3F00034F31004347371003473110434BA
:10002000F3F10F34F311043473720834731204348F
:10003000F3F20734F312043423A0070023A21700BD
:1000400023A4270023A6370023A8470023AA57008C
:1000500023AC870097120000938282FC1304F0FF08
:1000600073100434F3F5003473760034F3F60F3470
:1000700073770834F3F707347378003423A0B200A1
:1000800023A2C20023A4D20023A6E20023A8F200E8
:1000900023AA020123AC820097100000938000FA8B
:1000A000375A1632130A8A4973100A3473F0073428
:1000B000731A0A3423A0000023A240011715000080
:1000C000130545F4971500009385C5F7370610F022
:1000D0001306C6F26306B5028326C5002320D600A8
:1000E000832685002320D600832645002320D600C2
:1000F000832605002320D600130505016FF09FFD20
:10010000370510F0130505F223200500000000005C
:0401100000000000EB
:10100000FFFFFFFFFFFFFFFFFFFFFFFFFFFFFFFFF0
:10101000FFFFFFFFFFFFFFFFFFFFFFFFFFFFFFFFE0
:10102000FFFFFFFFFFFFFFFFFFFFFFFFFFFFFFFFD0
:10103000FFFFFFFFFFFFFFFFFFFFFFFFFFFFFFFFC0
:040000058000000077
:00000001FF
